:04000000C2014D29C3
:100008000800C216C21EC212C2190E28C215472005
:10001800031835280830A3005B20A20DA30B102875
:10002800C21E402065206120C21A35203A202208CD
:1000380003104829C216C21EC21242192828FE39C6
:10004800C300421503104829421A3028A600421658
:1000580047200318352826084E2003183528C21EC5
:1000680048294020652042114212C21146088400E6
:1000780044088417800446284608840044098005FB
:100088008417800508003A20652040206120430835
:10009800C2190138A2000830A300A20D03183A20A3
:1000A800031C402065206120A30B51283A206520BD
:1000B8004608840044080005FF3E470884004509B7
:1000C80043284708840045083D282C08A0002D082F
:1000D800A1000130A200A30164009B20031C882812
:1000E800A20B7028FF30A30703187028A007031C71
:1000F800A107031C4829FA30A2000030A300702889
:1001080064009B2003188428EC20A8010830A30071
:10011800ED209B200318A80AAB1EA801A20CA30B74
:100128008C28AB1AA213ED200314220808004608F5
:100138008400440884178004841300052B1B44069C
:10014800FF3E0800A4002908031403194829432185
:10015800031C0800A0002518831724088400200821
:1001680080008313A40AA903A728A60046088400D0
:100178008030C3050830A70003100318C30AD22033
:10018800A60CA70BC1280000AB1A430CD2204B21A8
:100198000314D2202F08A3002E08FD288413AB1FB8
:1001A800E128000844042B1F440680008417000837
:1001B8004404031C44068000ED2800084404031C82
:1001C80044062B1B44068000841744098005ED284B
:1001D80043172B081F39003EA1002A080E3E0318BA
:1001E800A10A431F0A294313A000023024210A2927
:1001F800A301A200FF30A207031CA307031C482980
:100208000330A100E6300A21FE28A101FC3EA0002F
:10021800A109031C1529FF300000A00703181029A5
:10022800A0076400A10F0F2908000310A00DA10D5D
:10023800FF3E03181929200848290310A10CA00C17
:10024800FF3E0318212920084829A20002302F293F
:10025800A20001302F29A80023082102031D3629F6
:10026800220820020430031801300319023028053F
:10027800031DFF3048290404031DFF30482984006A
:1002880031088A0030088200831303138312640044
:100298000800831607309F0099018312980183167E
:1002A8000230980006108610061188010710871082
:1002B80007118711071287128312F801F6010A3015
:1002C800F700FA01FF01FB018801871007110710E9
:1002D80086140611871664308A01FC2087120A30BA
:1002E8008A01FC2087160130A300F4308A01FD2022
:1002F8008A110A12992A07140A308A01092107105B
:10030800080087103E3088008A017F218614061174
:100318000130FB00640003307B028A110A120318C3
:10032800CF29B830FC006400C0307C028A110A1260
:100338000318BF2987108A017F21403088008A016D
:100348007F217C0888008A017F218714FD016400D1
:1003580040307D028A110A120318BA2988018A01DD
:100368007F21FD0A8A110A12031DAB29FC0A8A1192
:100378000A12031D972983108618831406198614F8
:10038800061D861083180615831C0611FB0A8A11A0
:100398000A12031D8E29861006158710B8308800AA
:1003A8008A017F21C03088008A017F21403088007F
:1003B8008A017F213F3088008A017F218614061137
:1003C800B83088008A017F21C03088008A017F21E7
:1003D800403088008A017F213F3088008A017F21D0
:1003E8008714861406110800871086140611013038
:1003F800FB00640003307B028A110A120318262AC4
:100408003E308800C03088008A017F214030880053
:100418008A017F21B83088008A017F213F30880017
:100428008A017F2183108618831406198614061DF5
:10043800861083180615831C0611FB0A8A110A12F6
:10044800031DFD298614061108007A0888008A0110
:100458007F21F60A64007608403C8A110A12031DBF
:10046800462A861006158710403088008A017F21A9
:10047800C03088008A017F21B8307E0788008A0151
:100488007F21871464007608803C8A110A12031DB4
:10049800682AFE0A64007E08083C8A110A12031DB5
:1004A800562AFE01F601861406118710403088008E
:1004B8008A017F21B8307E0788008A017F21C030F9
:1004C80088008A017F21871408007B08483E840041
:1004D8000008B200FF30A200A20A22080F3C8A11CD
:1004E8000A12031C982A8A110A12842232028A11DB
:1004F8000A12031D702A2208F8008A110A12982A83
:1005080002308A00220882073034313432343334DE
:100518003434353436343734383439346134623429
:10052800633464346534663408008A01F8218A012A
:1005380085210730C6004030C4002030AA00AB0136
:10054800AE01AF014C308A01B9206F308A01B92061
:1005580061308A01B92064308A01B92020308A01CB
:10056800B92069308A01B9206D308A01B92061301B
:100578008A01B92067308A01B92065308A01B9201B
:100588002E308A01B9202E308A01B9202E308A01F6
:10059800B9208A110A12A22B8A01F8218A01852121
:1005A800F601FE01F001F1017008A0007108A10038
:1005B8002030A30000308A012C218A110A12031D61
:1005C800992B0730C6001030C4000730C700083028
:1005D800C500A0308A01202071088A0120207008F7
:1005E8008A0120208A010520FA008A012922700840
:1005F800A0007108A1000430A30000308A0129215D
:10060800B2007008A0007108A1000830A3000030F3
:100618008A012921B4003208840034088A013F2164
:10062800B400B5007008A0007108A1000C30A30048
:1006380000308A012921B6003408350484003608C0
:100648008A013F21B600B7007008A0007108A10018
:100658001030A30000308A012921B8003608370479
:10066800840038088A013F21B800B9007008A0004A
:100678007108A1001430A30000308A012921BA00B2
:100688003808390484003A088A013F21BA00BB00BF
:100698007008A0007108A1001830A30000308A017A
:1006A8002921BC003A083B0484003C088A013F2108
:1006B800BC00BD007008A0007108A1001C30A30098
:1006C80000308A012921BE003C083D0484003E0810
:1006D8008A013F21BE00BF007008A0007108A10078
:1006E8002030A30000308A012921C0003E083F04C1
:1006F800840040088A013F21C000C100640040080E
:1007080041048A110A120319922B0F30A300A0305A
:100718008A01FD208A01F8218A018521F00A03193E
:10072800F10A8A110A12031DD82A0F30A300A0303B
:100738008A01FD208A01F8218A018521FC01FB013B
:10074800FD01F001F101F9012030F5000A30F70050
:10075800F001F101F601FE010730C6008030C40047
:100768002030AA00AB018A0184202A3C8A110A128F
:10077800031DB72B0930A9008430B000B101A501D1
:1007880068308A01A620FB01640009307B028A11C7
:100798000A120318082C7B08683E84000008B2007F
:1007A800FF30A200A20A22080F3C8A110A12031C79
:1007B800FE2B8A110A12EA2332028A110A12031D39
:1007C800D62B2208F8008A110A12FE2B03308A0061
:1007D80022088207303431343234333434343534F7
:1007E80036343734383439346134623463346434F9
:1007F800653466347B08683E840078088000FB0A0C
:100808008A110A12031DC82B6F08A000A101043029
:100818008A011C21B2002108B30070083204F700D5
:100828006908A000A10104308A011C21B200210836
:10083800B3006A083204F5006B08A000A101043077
:100848008A011C21B2002108B3006C083204F100AF
:100858006D08A000A10104308A011C21B200210802
:10086800B3006E083204F0007503F4007008F2005B
:100878007108F3006808FC0064007C08033C8A11D6
:100888000A120319EB2C64007C08013C8A110A1235
:100898000319572C64007C08023C8A110A120319B8
:1008A800D02A8A01AC2B0730C6008030C400203023
:1008B800AA00AB018830AC001330AD008A01692072
:1008C8008A110A12031CAC2B5D3C8A110A12031D03
:1008D800622C7508A9006930B000B101A501483043
:1008E8008A01A6208A110A12031CAC2BFB01FF30D7
:1008F8007507B200FF300318013EB3007B08A00063
:10090800A1013308A30032088A012C218A110A1296
:10091800031D9A2C8A0169227B08483E84007808C6
:100928008000FB0A8A110A12031D7B2CFB01FF3091
:100938007507B200FF300318013EB3007B08A00022
:10094800A1013308A30032088A012C218A110A1256
:10095800031DE92C7B08483E84000008B2003208D9
:10096800A000A10104308A011C21B2002108B300B3
:1009780001307B07B400B501B50D3408483E84004A
:100988000008B40034083204FA000730C6001030FA
:10099800C4000730C7000830C500A0308A012020F5
:1009A80071088A01202070088A0120207A088A01AB
:1009B8001E2005308A01FC20F00A0319F10A0230D2
:1009C800FB078A110A12031C9B2C8A01572C07303B
:1009D800C6008030C4002030AA00AB018830AC00CB
:1009E8001330AD008A0169208A110A12031CAC2B4E
:1009F8005D3C8A110A12031DF62C7508A90069309E
:100A0800B000B101A50148308A01A6208A110A1256
:100A1800031CAC2BFB01FF307507B200FF30031835
:100A2800013EB3007B08A000A1013308A3003208EF
:100A38008A012C218A110A12031D2E2D8A0169228E
:100A48007B08483E840078088000FB0A8A110A1255
:100A5800031D0F2DFB01FF307507B200FF3003188F
:100A6800013EB3007B08A000A1013308A3003208AF
:100A78008A012C218A110A12031D652D7B08483E24
:100A880084000008B2003208A000A10104308A01E5
:100A98001C21B2002108B30001307B07B400B50166
:100AA800B50D3408483E84000008B4003408320408
:100AB800FA008A0129220230FB078A110A12031C54
:0C0AC8002F2D8A01EB2C63008A01672DA2
:02400E00753DFE
:00000001FF
